:020000020000FC
:080000000C9499040C94E20336
:040014000C945304F1
:04001C000C947204CA
:040038000C9402041E
:040048000C94D10241
:100050000C94960210383810100010006C6C480098
:100060000000000000287C28287C28002038403030
:100070000870100064640810204C4C002050502080
:1000800054483400303020000000000010202020B0
:100090002020100020101010101020000028387CA4
:1000A000382800000010107C101000000000000034
:1000B000003030200000007C000000000000000044
:1000C00000303000000408102040000038444C5438
:1000D00064443800103010101010380038440418F0
:1000E00020407C003844043804443800081828486C
:1000F0007C0808007C404078044438001820407890
:10010000444438007C04081020202000384444383F
:10011000444438003844443C040830000000606027
:1001200000606000000030300030302008102040B7
:100130002010080000007C00007C00002010080453
:1001400008102000384404181000100038445C5493
:100150005C403800384444447C444400784444784B
:100160004444780038444040404438007844444493
:10017000444478007C40407840407C007C4040789B
:10018000404040003844405C44443C004444447C8B
:1001900044444400381010101010380004040404C3
:1001A0004444380044485060504844004040404077
:1001B00040407C00446C5444444444004464544CE7
:1001C0004444440038444444444438007844447827
:1001D0004040400038444444544834007844447813
:1001E0004844440038444038044438007C1010101F
:1001F00010101000444444444444380044444444EF
:1002000044281000444454545454280044442810B2
:10021000284444004444442810101000780810205A
:100220004040780038202020202038000040201056
:10023000080400003808080808083800102844009E
:100240000000000000000000000000FC3030100042
:1002500000000000000038043C443C00404078446A
:1002600044447800000038444044380004043C44CE
:1002700044443C000000384478403800182020787E
:100280002020200000003C44443C0438404070489A
:1002900048484800100010101010180008001808F6
:1002A0000808483040404850605048001010101076
:1002B00010101800000068545444440000007048B6
:1002C000484848000000384444443800000078445E
:1002D0004444784000003C4444443C04000058241A
:1002E00020207000000038403804380000207820BA
:1002F00020281000000048484858280000004444C6
:100300004428100000004444547C28000000484861
:10031000304848000000484848381060000078081D
:1003200030407800182020602020180010101000A5
:10033000101010003008080C080830002850000089
:100340000000000010386C44447C0000303132332F
:100350003435363738394142434445460C010203AF
:100360000405060708090A0B0C0102030405060729
:1003700008090A0B0000010001010001FF01FF0054
:10038000FFFF00FF0F931F9319D003D01F910F9110
:1003900008951FE000E442D01EE001E83FD011E0E4
:1003A00001E13CD008951FE000E438D011E001E104
:1003B00035D008951DE000E831D008951DE00027F4
:1003C0002DD0089500000000000000000000000093
:1003D000000000000895449A459A08953F933327FA
:1003E0003A9509F417C0B1F068D0ECDF02EA3DD0CD
:1003F000E9DF31D0A8F3012F38D0E4DF2CD080F32F
:1004000053D05BD003EA31D0DDDF25D048F33AD0BA
:10041000449A459A49D0802F3F9108953F933327BE
:100420003A9509F415C049D0CDDF0F9302EA1DD0EB
:10043000C9DF11D00F91A0F30F93012F16D00BD06D
:100440000F9170F30F9311D006D00F9148F3000075
:100450002BD03F9108953C98449A0894459AB2DF76
:10046000349B889445983C9A08953F9338E0449A89
:10047000000F08F04498459AA5DF45983A95B9F7DA
:100480003F9108953F933C98449A002738E0459A5D
:10049000089498DF349B8894001F459893DF3A9521
:1004A000B1F73C9A3F9108954498459A00000000A6
:1004B000449A00003C983D9808953C9A3D9A449A8D
:1004C000459A000000004498000000004598000094
:1004D000089510E41093C400F092C500F092C0009B
:1004E00018E41093C10016E01093C20003E10093DA
:1004F000D703E092DE03E2D008951091C1001069A5
:100500001093C100089513E01093C40011E01093FC
:10051000C50004E00093D703089510E41093C400CD
:10052000F092C50003E10093D70308950F930FB72E
:100530000F931F93FF93EF930091E1030F3F89F017
:100540000395EAE8F1E0E00FFF1D1081112321F48B
:100550000FEFE092DE0302C01093C6000093E103A8
:1005600019C0E091DF03F091E0030E2F0F2B49F04B
:10057000EF5FFF4F1491112339F4F092DF03F092F3
:10058000E003E092DE0306C01093C600E093DF03B1
:10059000F093E003EF91FF911F910F910FBF0F9127
:1005A00018950F930FB70F931F932F933F93FF93BC
:1005B000EF932091C6000091E203302F03950F774F
:1005C0001091E303011709F408C00093E203EAE085
:1005D000F2E0E30FFF1D20839160EF91FF913F91C7
:1005E0002F911F910F910FBF0F9118950F930091AD
:1005F000DE030023E1F3F092DE038093C6000F9147
:10060000089590FFFECF0F931F93FF93EF931091E8
:10061000E2030091E3038827011759F0EAE0F2E0D2
:10062000E00FFF1D808103950F770093E30301170F
:1006300009F49E7FEF91FF911F910F9108950F9301
:100640009E7FF092E203F092E3030F9108950F93DF
:10065000FF93EF930091DE030023E1F3F092DE03BA
:10066000E093DF03F093E00304910093C600EF9161
:10067000FF910F9108950F93FF93EF930091DE0385
:100680000023E1F3F092DE03F092E103EAE8F1E007
:100690000081002331F40FEF0093E103E092DE03C9
:1006A00002C00093C600EF91FF910F910895882733
:1006B00090FD839508958091DE0308950FEF0093D8
:1006C000E103F092DF03F092E0030895BF93AF934C
:1006D000A8E3B1E016E02D913D91232B31F018965F
:1006E0001A95C9F7EF91FF9111C0ED93FD93ED922B
:1006F0000D93EF91FF9101910D9301910D930D9247
:100700001D921A973297ED93FC93119708950A2E34
:100710000B2A69F0FF93EF93ED91FD9114960D91E3
:100720001D9101931193189703D0EF91FF910895B4
:100730000AE0FD920A95E9F7089517E0A8E3B1E011
:10074000F7DF1A95E9F70895A8E3B1E026E0BF9333
:10075000AF930D911D91012B21F012972F9307D08C
:100760002F91AF91BF911A962A9589F708950D910F
:100770001D9112962D913C913F3F19F03A953C9373
:1007800071F0322F3E253E93222311F0149601C0C2
:1007900012972D913D91D8012D933D9306C0159749
:1007A000FF93EF93B4DFEF91FF9108955A9A0E945F
:1007B000C20102E00093690001D00895E89A08950B
:1007C000E89808950F930FB70F9394600F910FBFA0
:1007D0000F9118950F93F4BC05E005BD0FE707BD19
:1007E0000F9108950DE70093E4030895F092E40358
:1007F00002E005BB02E000936E00089500E0009364
:100800006E0008950F93F6BC78940FB70F931F9363
:100810000091E403002339F00A950093E40319F4EE
:100820009860F092E9030091EA03000F1E2D4F9BA0
:100830001127012B0093EA03003869F40091E903C2
:100840000E15D9F00091E80304600093E803E092EC
:10085000E903C8DF12C00F3721F00F3F71F412D047
:100860000CC00091E903002341F09062F092E9038B
:100870000091E8030B7F0093E8031F910F910FBFD6
:100880000F911895BBDF01D0089500E800936D002B
:1008900004E000936800089500E000936D0000E01C
:1008A0000093680008950F930FB70F93F5DF9EDF55
:1008B0000F910FBF0F9118950F93F092B00007E0C2
:1008C0000093B10003EC0093B30002D00F910895A0
:1008D00002E007BB02E000937000089500E000937F
:1008E000700008950F930FB70F93F092B20000912C
:1008F000EB03002329F00A950093EB0309F49260BF
:100900000091DB030A9511F4906409E10093DB0385
:100910000F910FBF0F911895A89504B7077F04BFDB
:100920000091600008610093600000270093600060
:100930000895F2DF2227E0E0F1E014E000272193A0
:100940000A95E9F71A95D1F7FF24EE24E394992745
:10095000882499240FEF0093EA03F092D50309E16C
:100960000093DB0305E00093DD0334DFAAD133DD20
:1009700037D23DD28ADFA0DFE0DEBED097D0A9D04B
:10098000A8DD70D30091D703043009F4BCDD46D252
:10099000EBD10ED20BDF78940E94B6070E9462085A
:1009A0000E947D021CC01AD195FF07C09F7D009157
:1009B000D6030E250093D60385D390FF14C0009173
:1009C000D603002311F0E4D2EECFFED008E20F935D
:1009D0000E94F8040F9190FF02C00A95C1F70EE63D
:1009E0000093EB03E0CF91FFDECF9D7FBBD0DBCF49
:1009F00008DE8F313AF5883041F40091D5030023A9
:100A0000C9F10A950093D50335C08D3041F40091AA
:100A1000EE03002309F02FD0E092EE032BC08930C3
:100A200011F480E211C08A3031F497FD24D090682F
:100A3000F092EE031FC08F938EE506D08F91805CFD
:100A40000C942405E7FC16C097FD15D00091EE0329
:100A5000002321F0F092EE03F092D50374D00091C0
:100A6000D503A00FBF1D8D9303950093D5030431CB
:100A70000CF0906808950091D40303950D3014F0A4
:100A80004DD00CE00093D4035ED006D0F092D50395
:100A90009F77F092EE0308950F9304E110E21D9307
:100AA0000A95E9F7FD9211960F9108950DE0AAE8D5
:100AB000B2E0F2DF0A95E9F708950F9304E11D9380
:100AC000139517FD10E20A95D1F7FD9211960F913B
:100AD0000895E4E4F1E1AAE8B2E00590002011F005
:100AE0000D92FBCFE092D4030BE0A6EBB2E011E352
:100AF000E4DF0A95E9F708950DE0AAE8B2E0E0E046
:100B0000F1E01DEE2FEF37E0A193B19355962D93B1
:100B10003193119312510A95B9F70895E0E0F1E08D
:100B20000190119032971CE0A4E0B1E00D91019387
:100B30000D910193129632961A95C1F70192119276
:100B4000D001AADF08950091D4030D300CF00027E6
:100B5000000F000FE0E0F1E0E00FFF1DA191B19167
:100B600032970895E091EC03F091ED030E2F0F2BD7
:100B700051F5E9DFEEEBF3E00D9101930023E1F78E
:100B8000EEEBF3E00091D503043114F003E109C06A
:100B900097FF07C00091D503002319F00A95009331
:100BA000D503E00FFF1D0FE50083CDDF0D01DF0151
:100BB000F0010EEB13E008010FEF88DDA093EC03CA
:100BC000B093ED0308950895A091EC03B091ED0367
:100BD0009EDDF092EC03F092ED0308951FD092FF9A
:100BE00002C09AD09B7F96FF03C00E94A4039F7B04
:100BF00094FF09C00091DD030A9511F4FBD005E0D4
:100C00000093DD039F7E08950F938F93FF93EF93DF
:100C1000E5DFEF91FF918F910F910895A0E0B1E092
:100C20002EE044E550E0ED91FD91BD90CD900E2E6B
:100C30000F2A29F00191002311F004D0FBCF2A954F
:100C400091F708950F0107FD23C0015208F15D9847
:100C5000E02FFF27EE0FFF1FEE0FFF1FEE0FFF1F0E
:100C6000E40FF51F68E06590882767FC38D083950E
:100C700066FC35D0839565FC32D0839564FC2FD01B
:100C8000839563FC2CD0839562FC29D06A9559F733
:100C90005D9AF00102D0B00E0895093111F407E019
:100CA00005C0003811F404E001C00CE008950A33D7
:100CB00011F407E005C0003811F404E001C00CE0B5
:100CC0000895209A219A229A239A389A399A3A9A20
:100CD0003B9A539A549A559A5D9A5C9A0895382E85
:100CE000462E880F880D8B0D660F690D6C0D05D093
:100CF000639503D0642D832D08955B98282E28B822
:100D0000229425B85C985C9A5B9A262E28B8229487
:100D100025B85C985C9A089566D01091D803139515
:100D20001093D8031C33DCF09061F092D80310913B
:100D3000D90313951093D9031C338CF01091E80359
:100D400012601093E803F092D9031091DA0313951F
:100D50001093DA0318311CF0F092DA0300C004D0CB
:100D600008955CD001D00895AEE7B1E00091DA03B8
:100D7000ECE5F3E0E00FFF1D049117D00AE30D93BB
:100D80000091D90312D00AE30D930091D8030DD03E
:100D900000E80D9311E40091DA030C300CF010E53B
:100DA0001D931DE41D93FD920895802FA2D00895F8
:100DB000A4E3B1E0EEE7F1E0ED93FD9304D00D93F1
:100DC00000E00D93089522270191002329F06FDFA1
:100DD000200FD0F7002703C00FEF021B06950895E0
:100DE000569A5E9808954E9A08955E980895579879
:100DF0005F9A08950091DC030F3F79F0FF93EF9322
:100E0000E4E7F3E0039507700093DC03000FE00FC5
:100E1000FF1D85909490EF91FF9108958F9312E0BC
:100E2000DDDA8F7741D08C330CF088278093D8039C
:100E300013E0D4DA8F7738D08C330CF08827809386
:100E4000D90314E0CBDA8F732FD088310CF08827C8
:100E50008093DA038F9108958F93082F0C3328F431
:100E60008093D8032BD012E0D9DA8F910895082F00
:100E70000C3328F48093D90321D013E0CFDA0895FE
:100E8000082F083128F48093DA0318D014E0C6DA6A
:100E90000895222738E0000F221F211710F0039534
:100EA000211B3A95C1F708958F9382958F700AE0C0
:100EB000809F002D8F918F70800F0895082F04D090
:100EC0000295022B802F08951AE0E3DF0770089542
:100ED000FF93EF93ECE4F3E0E80FFF1D8491EF91B3
:100EE000FF910895813624F08B3710F400E2801BC7
:100EF0000895E4DF8F9382958F70EADF8D938F9151
:100F00008F70E6DF8D930895A1BDB2BD119611FDDE
:100F1000FA9A1FBBF999FECF00B508950F9300917F
:100F2000D8038EE1080F0C330CF00C53C0DB882380
:100F300031F46ADE8091D803081729F0F7CF61DB1E
:100F4000D1DF0F91089588E50F9108958F93B3DB5A
:100F5000882311F459DEFBCF8F9148DB0895ABDB7A
:100F6000882311F451DEFBCF72DB08958F93A3DB4E
:100F7000882311F449DEFBCF8F91E8EFF1E167CBD5
:100F8000089599DB882311F43FDEFBCF74DB0895CD
:100F900038DBA8DF883509F075C0E0EAF1E1DFDF72
:100FA000BDDFD4DFE3DF843541F0833431F18234B7
:100FB00041F1883509F41DC0F0CFEEEAF1E164D0CB
:100FC000B0F05EDFD3DFE0ECF1E15ED080F04FDF28
:100FD000CDDFE2EDF1E158D050F03EDF0091D803D3
:100FE0000A950093D8030E948C06C0DF4BC00E9474
:100FF000B106E4EEF1E1B3DF45C0ECEFF1E1AFDFC4
:1010000041C00091D703043021F4E8E3F2E103E1A9
:1010100005C00331D1F4EEE1F2E104E00093D7031F
:101020009EDF0091D80383E0080F0C330CF00C53C3
:10103000EBDD8091D8030817D9F708D00091D703CA
:10104000043011F06ADA01C05EDA1CC0BF93AF93BE
:101050000091D703ADEFB1E000BD16E055DFAF91D1
:10106000BF910895BF93AF93ADEFB1E011E04CDFB6
:10107000043019F0033109F003E10093D703AF9175
:10108000BF9108952FD008956ADF48DF5FDF88356C
:1010900011F4089408950DD0C0F3082F3FDF56DFF8
:1010A0008835B9F306D0D0F31AE0019F800D8894FB
:1010B0000895803328F08A3318F480538894089573
:1010C00008940895EAE5F1E14ADF002720D0ECE733
:1010D000F1E10091D603002311F0EEE8F1E13FDFEA
:1010E00045DF0895EAE5F1E13ADF002710D03EDF61
:1010F00008958091DA03FDDE8AE38D938091D90310
:10110000F8DE8AE38D938091D803F3DE0895D3DA75
:10111000882311F479DDFBCFFF93EF93BF93AF9357
:101120000F93AAE8B1E0E5DF0F91002321F08DE0F5
:101130008D938AE08D93FD929EDAAF91BF91EF91EE
:10114000FF910895447574636874726F6E697820B6
:101150005465726D696E616C0000415652204F7388
:1011600063696C6C6F73636F7065205465726D6931
:101170006E616C2056332E3061200000204D6F646C
:1011800065206973205465726D696E616C00204D35
:101190006F646520697320436F6D6D616E6400003C
:1011A000436F6D6D616E6428542C42293A003220E1
:1011B000646967697420686F7572733A2020200033
:1011C00032206469676974206D696E757465733A5D
:1011D000200032206469676974207365636F6E64F0
:1011E000733A200043616E63656C206F722054690E
:1011F0006D656F75742000000D0A0000436F7079F3
:101200007269676874203230303820204A616E205D
:10121000502E4D2E206465205269650D0A005377CB
:1012200069746368696E6720746F203438303020C9
:1012300042617564200D0A00537769746368696EB2
:101240006720746F20313932303020426175640D6F
:021250000A0092
:00000001FF
